:10000000BD29FF3FFF3F00000000080021308312A0
:10001000CD00CD0B092808000F308312CC004730EB
:10002000CD00CD0B1128CC0B1128000000000800DA
:100030008312B21B1D2806131E280617321B222806
:10004000861223288616B21A272806122828061692
:10005000321A2C2886112D288615281831280614C6
:1000600032280610061503200611B2193928061386
:100070003A28061732193E2886123F288616B218EB
:1000800043280612442806163218482886114928A3
:10009000861528184D2806144E280610061503202C
:1000A0000611281C55280C2056280620080083120B
:1000B00028103108B20018202814080083122208E2
:1000C0008A002108820008008312C4018C01C20149
:1000D000083042020318B428C30105187A28C30A5D
:1000E0004308643C0318772801308C007A2800000C
:1000F00000006D281330CD00CD0B7C2800000000DF
:10010000051894284208073CC0004008C10001308F
:10011000C000410803199028C00D4010FF3E8A28F6
:10012000C0094008C405B2284208073CC000400886
:10013000C1000130C00041080319A228C00D4010C1
:10014000FF3E9C284008C404C301051CB228C30A12
:100150004308643C0318AF2801308C00B22800002B
:100160000000A528C20A68284408C00008008316B9
:100170000611061086110612861206138312061146
:10018000061006138612061286110C200C200C2075
:10019000061686150615032006110C2006150320E9
:1001A00006110C200615032006110C2086110615D9
:1001B000032006110C20061503200611061206174F
:1001C0000615032006110C200613861506150320BC
:1001D000061186110615032006110C2006150320B2
:1001E000061186150615032006110C20861106152A
:1001F0000320061106178616061686150615032017
:1002000006110C202814080006308312CB0013308E
:10021000CC00AD30CD00CD0B0B29CC0B0B29CB0B7B
:100220000B2900000000080083120313C801C90154
:100230001030CC00410DC80DC90D4408C802450856
:10024000031C450FC90203182C294408C807450898
:100250000318450FC9070310C00DC10DCC0B1A2997
:1002600008001A308312CD00CD0B34290000051888
:1002700046293530CD00CD0B3B29051C46292130C0
:10028000CD00CD0B41290130C0004629080083165E
:100290000510831205104130CC00EE30CD00CD0B9F
:1002A0004F29CC0B4F29000005141330CD00CD0B86
:1002B0005729000000008316051408006F298030BC
:1002C0008312AD008029C030AD0080299430AD008C
:1002D0008029D430AD0080298030AD0080292D08E0
:1002E000013A03195F292D08023A031963292D08E1
:1002F000033A031966292D08043A031969296C2960
:100300002E03C0002D08C0074008AD004008B20011
:1003100018202810B00130082F07840000080319A6
:10032000992930082F0784000008B1005720B00A2F
:100330008B292814080083122E08A1002F08A20080
:100340005E208A110A12C1004108003C0318B92935
:100350002E08A1002F08A2005E208A110A12C000F8
:100360002D08840040088000AD0AAE0A0319AF0AC8
:100370009B292D0884008001080083168601013026
:1003800085008312850183160510831205108316DC
:100390008511831285118C018D018E0180300E062E
:1003A000C00080304002031DD72906300D0203181B
:1003B000E12985110421851504218D0A03198E0A6E
:1003C000CE29B7200130B20018200C30B20018201E
:1003D0000F30AD006D30AE000330AF009B21013017
:1003E000AD000130AE000F30AF005E210F30AD0028
:1003F0007E30AE000330AF009B210230AD000130F3
:10040000AE000F30AF005E210F30AD008F30AE0078
:100410000330AF009B210330AD000130AE000F3040
:10042000AF005E21042104210130B20018204721D1
:10043000312140080319282B64204008A3006420C0
:100440004008AA0064204008AB0064204008AC00CB
:1004500064204008A9000C0803193D2A0F30AD00A4
:10046000B030AE000330AF009B210130AD00013051
:10047000AE000F30AF005E21272B2A082307C000F3
:10048000C1010318C10A2B08C0070318C10A2C08B0
:10049000C0070318C10AFF304005C2004108C3006D
:1004A0000030C30500304306031D582A42082906C0
:1004B000031D192B0F30AD004B30AE000330AF00E1
:1004C0009B212308A400A5012408A500A4012A0853
:1004D000A4040030A5042B08A600A7012608C1002B
:1004E000C0012C084004C2004108C3000030C3040E
:1004F0004208A6004308A7004308803C031D822A47
:100500004208003C03188B2A2D309500FF30A605C9
:100510007F30A7058D2A203095006430C40000305C
:10052000C5002608C0002708C10014210A30C400F5
:100530000030C50014214808C0004908C10030300F
:10054000400796000A30C4000030C5002608C000ED
:100550002708C10014210A30C4000030C50014214E
:100560004808C0004908C1003030400797000A30F1
:10057000C4000030C5002608C0002708C1001421AF
:100580004808C0004908C100303040079900DF30FA
:100590009A000130AD000130AE000F30AF005E2197
:1005A0000F30AD005C30AE000330AF009B216430F3
:1005B000C4000030C5002408C0002508C100142173
:1005C0000A30C4000030C50014214808C0004908A2
:1005D000C1003030400796000A30C4000030C5002A
:1005E0002408C0002508C10014210A30C4000030CE
:1005F000C50014214808C0004908C1003030400738
:1006000097000A30C4000030C5002408C000250847
:10061000C10014214808C0004908C100303040071B
:1006200099000230AD000130AE000F30AF005E2106
:10063000272B0F30AD00A030AE000330AF009B2160
:100640000230AD000130AE000F30AF005E21372B1D
:100650000F30AD003A30AE000330AF009B210230C6
:10066000AD000130AE000F30AF005E210421042147
:10067000172A392B50346134733420346434653490
:1006800020347234653470346F346E3473346534AE
:100690002E342E340034543465346D3470342034A8
:1006A0003D342034303430342E343034203443342C
:1006B0002034203420340034523448342034203460
:1006C00020343D342034303430342E34303420342F
:1006D0002534203420342034003444344834543415
:1006E00032343234203431343634463438343434CD
:1006F000203438344D3448347A3400344D3469343D
:100700006B3472346F344334203437342E343634FF
:1007100030342034503472346F3420340034563442
:1007200065347234733469346F346E342034313448
:1007300033342D34303437342D34323434340034BF
:1007400043346834653463346B34733475346D34D6
:1007500020344534723472346F34723421340034AE
:10076000543469346D34653420346F3475347434E2
:1007700021340034FF3FFF3FFF3FFF3FFF3FFF3F7C
:02400E00F13F80
:020000040000FA
:104200007000610075006C0066006A0075006A004D
:104210006F000D000A000000FF00FF00FF00FF001C
:104220004D0069006B0072006F00430020005000D9
:1042300072006F00200037002E00360030000000B2
:104240005500410052005400330020003900360070
:10425000300030006200640073000D000A000000AE
:104260007200650076002000310033002F0030001E
:104270002F0032003000320034000D000A00000030
:00000001FF
